:1000000012C01895B9C21895189518951895189595
:100010001895189518951895189518951895189578
:100020001895189518958FE58DBFC0E4E8E34E2E1E
:1000300084E08EBFD4E0F4E05F2EEEEFF3E0A0E6C4
:10004000B0E088278D933197E9F7B7D46624899A71
:10005000A0988B98BC98BD98A89A939AC49AC59A70
:100060008D9ABF9A8E9A9598C7989698E1E0F0E09D
:10007000A0E1B0E0ACD50F3609F01AC0E2E0F0E044
:10008000A1E6B0E0A6D5E0E0F0E0AEE6B0E09FD5B6
:10009000E4E0F0E0A1E7B0E09AD5E5E0F0E0A2E727
:1000A000B0E097D5E7E0F0E0A4E7B0E092D544C037
:1000B000E1E0F0E0A0E1BB278FE68C937BE776D50B
:1000C0008AEC93E0A1E6B0E08D939C9381E080936D
:1000D0006E00E2E0F0E0A1E6B0E07BE769D5E0E0A9
:1000E000F0E0AEE6B0E07BE761D581E0809371009F
:1000F000E4E0F0E0A0E1BB2781E08C937BE756D5FC
:100100008CEA93E0A2E7B0E08D939C93E5E0F0E009
:100110000CEA13E0A0E1BB277BE74AD580E194E03D
:10012000A4E7B0E08D939C93E7E0F0E000E114E0F9
:10013000A0E1BB277BE73CD5789485B7837F85BF5B
:100140008BB780688BBF80E0809360000091710066
:10015000013009F002C0919A01C091985BD3D8D3C5
:100160008CE073D410D4E2EEFBE005D40AD4E4EFC3
:10017000FBE001D48CED95E094D405D40027A3E3F3
:10018000B0E08C9180FB0EF401E041E0041708F030
:1001900070C1E6E0FCE0EFD38FEB11E003D4E8E1BF
:1001A000FCE0E9D3A0E2B4E0E3E6F0E0AFD4DBD3D7
:1001B000EEE1FCE0E0D3A0E2B4E0E4E6F0E09FD4BE
:1001C000D2D3E0E2FCE0D7D300916000003009F028
:1001D00088C00027A3E3B0E08C9180FB0EF401E01F
:1001E00041E0041708F039C0A1E6B0E00D911C9180
:1001F00041E050E0040F151FA1E6B0E00D931C9301
:10020000A1E6B0E00D911C91083354E0150714F0FD
:1002100009F001C006C08BE693E0A1E6B0E08D9343
:100220009C9376D38FEB11E0BDD3E8E1FCE0A3D340
:10023000A0E2B4E0E3E6F0E069D495D3EEE1FCE0BF
:100240009AD3A0E2B4E0E4E6F0E059D48CD3E0E243
:10025000FCE091D38AEA90E024D40027A6E3B0E042
:100260008C9185FB0EF401E041E0041708F038C0E2
:10027000A1E6B0E00D911C9141E050E0041B150B8C
:10028000A1E6B0E00D931C93A1E6B0E00D911C91A6
:100290000B3653E015070CF401C006C088E394E068
:1002A000A1E6B0E08D939C9333D38FEB11E07AD32A
:1002B000E8E1FCE060D3A0E2B4E0E3E6F0E026D4BD
:1002C00052D3EEE1FCE057D3A0E2B4E0E4E6F0E084
:1002D00016D449D3E0E2FCE04ED38AEA90E0E1D3C1
:1002E00073CFA1E6B0E08D919C91A2E7B0E08D9331
:1002F0009C93E5E0F0E0A1E6B0E07BE759D443D37E
:10030000EAE2FCE038D38FEB11E04CD3E8E1FCE00B
:1003100032D3A0E2B4E0E3E6F0E0F8D324D3EEE198
:10032000FCE029D3A0E2B4E0E4E6F0E0E8D31BD39C
:10033000E0E2FCE020D300916000013009F088C0C9
:100340000027A3E3B0E08C9180FB0EF401E041E0D4
:10035000041708F039C0A1E6B0E00D911C9141E00E
:1003600050E0040F151FA1E6B0E00D931C93A1E629
:10037000B0E00D911C91083354E0150714F009F01A
:1003800001C006C08BE693E0A1E6B0E08D939C939C
:10039000BFD28FEB11E006D3E8E1FCE0ECD2A0E2A3
:1003A000B4E0E3E6F0E0B2D3DED2EEE1FCE0E3D28B
:1003B000A0E2B4E0E4E6F0E0A2D3D5D2E0E2FCE0D3
:1003C000DAD28AEA90E06DD30027A6E3B0E08C9100
:1003D00085FB0EF401E041E0041708F038C0A1E607
:1003E000B0E00D911C9141E050E0041B150BA1E61B
:1003F000B0E00D931C93A1E6B0E00D911C910B367B
:1004000053E015070CF401C006C088E394E0A1E6B0
:10041000B0E08D939C937CD28FEB11E0C3D2E8E1E6
:10042000FCE0A9D2A0E2B4E0E3E6F0E06FD39BD217
:10043000EEE1FCE0A0D2A0E2B4E0E4E6F0E05FD3BD
:1004400092D2E0E2FCE097D28AEA90E02AD373CF1E
:10045000A1E6B0E08D919C91A4E7B0E08D939C93D0
:10046000E7E0F0E0A1E6B0E07BE7A2D380E0809394
:100470006000E2E0F0E0A1E6B0E0ABD3CBD148D23F
:1004800015D200916000013009F001C0B4D00027FE
:10049000A6E3B0E08C9184FB0EF401E041E0041788
:1004A00008F021C000917100003009F00DC081E01A
:1004B00080937100E4E0F0E0A0E1BB2781E08C9341
:1004C0007BE774D3919A0CC080E080937100E4E0E4
:1004D000F0E0A0E1BB2780E08C937BE767D39198A5
:1004E00088EC90E0DED20027A3E3B0E08C9180FBA3
:1004F0000EF401E041E0041708F019C0A2E7B0E0F3
:100500008D919C91A1E6B0E08D939C93E2E0F0E0A8
:10051000A2E7B0E07BE74CD37DD1FAD134D2E6E05C
:10052000FCE029D2E1E0F0E03FD22DD2BFD100279C
:10053000A6E3B0E08C9185FB0EF401E041E00417E6
:1005400008F019C0A4E7B0E08D919C91A1E6B0E05D
:100550008D939C93E2E0F0E0A4E7B0E07BE728D342
:1005600059D1D6D110D2EAE2FCE005D2E1E0F0E0C8
:100570001BD209D29BD185CF0F921F922F923F920F
:100580004F925F927F92AF92BF920F931F932F93E0
:100590003F934F935F936F937F938F939F93AF930B
:1005A000BF93CF93DF93EF93FF938FB78F93A0E623
:1005B000B0E08C918F5F8C9388EC90E072D28F9139
:1005C0008FBFFF91EF91DF91CF91BF91AF919F913D
:1005D0008F917F916F915F914F913F912F911F91DB
:1005E0000F91BF90AF907F905F904F903F902F9072
:1005F0001F900F901895C7D1ECE3FCE0BCD1E1E06F
:10060000F0E0D2D1C0D1EEE4FCE0B5D18FEB11E047
:10061000C9D1E8E1FCE0AFD1A0E2B4E0E3E6F0E06C
:1006200075D2A1D1EEE1FCE0A6D1A0E2B4E0E4E60F
:10063000F0E065D298D1E0E2FCE09DD1009160004D
:10064000013009F088C00027A3E3B0E08C9180FB63
:100650000EF401E041E0041708F039C0A1E6B0E073
:100660000D911C9141E050E0040F151FA1E6B0E090
:100670000D931C93A1E6B0E00D911C91083354E05A
:10068000150714F009F001C006C08BE693E0A1E65F
:10069000B0E08D939C933CD18FEB11E083D1E8E1E6
:1006A000FCE069D1A0E2B4E0E3E6F0E02FD25BD158
:1006B000EEE1FCE060D1A0E2B4E0E4E6F0E01FD2BD
:1006C00052D1E0E2FCE057D18AEA90E0EAD100277B
:1006D000A6E3B0E08C9185FB0EF401E041E0041745
:1006E00008F038C0A1E6B0E00D911C9141E050E067
:1006F000041B150BA1E6B0E00D931C93A1E6B0E03E
:100700000D911C910B3653E015070CF401C006C087
:1007100088E394E0A1E6B0E08D939C93F9D08FEB51
:1007200011E040D1E8E1FCE026D1A0E2B4E0E3E64C
:10073000F0E0ECD118D1EEE1FCE01DD1A0E2B4E094
:10074000E4E6F0E0DCD10FD1E0E2FCE014D18AEA8B
:1007500090E0A7D173CF17D1EEE5FCE00CD18FEB81
:1007600011E020D1EEE6FCE006D1A6E6B0E0FDD037
:10077000E2E7FCE000D100916000023009F02FC0F8
:100780000027A3E3B0E08C9180FB0EF401E041E090
:10079000041708F00CC081E080936E008FEB14E02A
:1007A00001D1E6E7FCE0E7D088EC90E07AD10027C1
:1007B000A6E3B0E08C9185FB0EF401E041E0041764
:1007C00008F00CC080E080936E008FEB14E0EAD05C
:1007D000EEE7FCE0D0D088EC90E063D1CCCFD3D072
:1007E000E6E8FCE0C8D0E0E0F0E0AEE6B0E07BE7B1
:1007F000DDD1E2E0F0E0A1E6B0E07BE7D9D180E036
:1008000080936000E1E0F0E0CFD0BDD003D080D095
:100810004DD0089500916E00013009F00DC0A1E6A1
:10082000B0E00D911C9140E058E4042B152BAFE68D
:10083000B0E00D931C930CC0A1E6B0E00D911C91AB
:1008400040E050E4042B152BAFE6B0E00D931C9371
:100850009598969ABF9A8D9A9598AFE6B0E090E1F8
:100860008D91983018F4392F992702C038E09850AC
:100870008795C79808F4C79A00000000959AEF93EF
:10088000FF93E0E1F0E001D1FF91EF919598EF93B4
:10089000FF93E0E1F0E0F9D0FF91EF913A9541F755
:1008A0009923F1F696989598C798089500916E004F
:1008B000013009F006C0A6E6B0E0E6E7FCE000D1B2
:1008C00005C0A6E6B0E0EEE7FCE0FAD08FE711E065
:1008D00069D0A0E2B4E0E3E6F0E018D144D0EEE164
:1008E000FCE049D0A0E2B4E0E4E6F0E008D13BD07F
:1008F000E8E9FCE040D0A6E6B0E037D0EEE9FCE065
:100900003AD08FEB11E04ED0E2EAFCE034D008950B
:10091000A1E6B0E08D919C91A4E6B0E08D939C930C
:1009200080E080936300A4E6B0E00D911C91093053
:1009300050E0150714F009F001C012C0A3E6B0E0C2
:100940008C918F5F8C93A4E6B0E00D911C914AE0EE
:1009500050E0041B150BA4E6B0E00D931C93E3CF0D
:100960000895F894FFCFA0E2B4E08D91882311F0B0
:1009700066D0FBCF0895A9D0802D11F060D0FBCFB9
:10098000089580EC62C081E060D014D080E85DC042
:100990008FE7213039F08FEB223021F08FE82330C0
:1009A00009F08FEC810F51C088EE93E07AD0319737
:1009B000D9F7089583E0992774C08AEF90E071D049
:1009C000889AA59AA49AA39AA29AA19AA99885E02E
:1009D00090E067D0AA989098AD98AC9AAB9AAA9AF2
:1009E000EF93FF93E0E6F0E050D0FF91EF91AA98EB
:1009F00055D0AA9AEF93FF93E0E6F0E046D0FF913E
:100A0000EF91AA984BD0AA9AEF93FF93E0E6F0E01B
:100A10003CD0FF91EF91AA9841D0AB98AA9AEF935E
:100A2000FF93E0E6F0E031D0FF91EF91AA9836D045
:100A300088E20BD08EE009D086E007D00895A99A0D
:100A4000829505D004D02AD00895A998F9CF85952C
:100A500010F4AB9A01C0AB98859510F4AC9A01C024
:100A6000AC98859510F4AD9A01C0AD98859510F4B9
:100A7000909A01C09098AA9AEF93FF93E0E6F0E075
:100A800004D0FF91EF91AA9808953197F1F7089556
:100A9000689462F80895E89462F8089581E090E01F
:100AA00000C0EF93FF93EE27E82BE92B31F0E8EE3F
:100AB000F3E03197F1F70197D1F7FF91EF910895A6
:100AC00004D00D920020E1F70895C89531960020DA
:100AD0000895000F111F221F331F089500951095D0
:100AE000209530950F5F1F4F2F4F3F4F0895019175
:100AF00010810EC001911191219130810BC00191A3
:100B0000108117FF05C03FEF2FEF04C000811127B0
:100B10002227332737FF03C0E1DF8DE28D93CF9388
:100B2000DF93CF92DF92EF92AA24BB24CC24DD2462
:100B3000EE2440E2CAE0DD2755E093E38881890F87
:100B400087FD9F7083FD907F891B89935A95A9F734
:100B5000C0DFAA1CBB1CCC1CDD1CEE1C4A9551F747
:100B6000E894EFE0FF2782910ED0EB30E0F71EF023
:100B700068948A2D0CD088278D93EF90DF90CF90CA
:100B8000DF91CF910895982F829501D0892F8F7092
:100B9000805D26F0803309F4089568948D9308955C
:100BA000E199FECFEEBBFFBB3196089591E001C005
:100BB00092E07B3751F47FB7F894F2DF8D918DBBD3
:100BC000E29AE19A9A95C9F77FBF7727089591E055
:100BD00001C092E0E5DFE09A8DB38D939A95D1F74D
:100BE000089520464D207472616E736D697474654A
:100BF000722000007777772E6E6F76612D746563B3
:100C0000682E6875000020202020202043482E31C7
:100C10002020202020200000203C3D2000002E002D
:100C20004D487A20203D3E2000002020202020201A
:100C300043482E3220202020202000002020202089
:100C400053657474696E6773202020200000313A68
:100C5000204672657175656E637920200000323A16
:100C600020417564696F206D6F64652020003C3DF4
:100C70002000203D3E002053746572656F00204DBA
:100C80006F6E6F2020002020202020536176656445
:100C900020202020202000004D487A200000202025
:100CA000200020464D205472616E736D6974746526
:040CB00072200000AE
:00000001FF
